:020000040000FA
:0A00000000000000EDEF00F0FDD05D
:080018004AD10E500C6E1218C3
:10002000186E0D50D8A411503AE00D267E0E03E351
:100030000D5E03E336D00D5E31E310C00AF00FC051
:100040000BF00C8E128E106A0F6A0E6A180E176E65
:100050000C320B320A3206E31450102613500F22D2
:1000600012500E220E320F321032172EF1D70EBE62
:1000700007D010360F360E360D5210E00D060C3438
:1000800016E3103E14D00F3E12D00E3E10D0D88092
:100090000E320F3210320D3E0AD003D016840D6A94
:1000A00002D016820D68106A0F6A800E0E6E18AEAE
:1000B0000E9E105012000DC017F00E5010C00EF022
:1000C000106E103617321032166A1036173602E3E9
:1000D0001684167E06E11680176A106A0F6A0E6A89
:1000E0000BD0172803E0D880103206D0D8901032F9
:1000F00002E1168201D0168616B604D016A20FD0E1
:1001000016B407D07F0E106EFF0E0F6E0E6E0D6EC2
:1001100023D0800E106E01D0106A000EF6D716B0F4
:10012000FBD70D6A9F0E1760EBD77E0E1764F4D7CE
:100130009E0E175C07E0D89010320F320E320D324F
:10014000172AF6D716A408D0D880000E0D560E56E2
:100150000F56105610AEE0D70D5012000F6A106AFD
:10016000189E0AD0189E10AE07D0D880000E0D56EB
:100170000E560F561056188E960E176E105209E036
:10018000080E17260EC00DF00FC00EF010C00FF0B5
:1001900011D00F520FE1080E175E0E5007E1080E46
:1001A000175E0D5002E1105010D00D6A0F6E0DC099
:1001B0000EF00D6A0FBE06D0D8900D360E360F36F3
:1001C0001706F8D718AE0F9E17500DC010F00D6E21
:1001D0000F500EC00FF00E6E1200400E166E4F0E36
:1001E000AF6E240EAC6E900EAB6E0001C69AC00EC0
:1001F000926EE00E936EC00E946E0F0EC16E070EDF
:10020000B46E6FD0F2A403D0F294817A11009EAA4A
:1002100019D0060EAB1412E1E2CF1AF0E1CF19F0BB
:100220001B2A11EE00F01B50E126000EE222AECF99
:10023000E7FF1AC0E2FF19C0E1FF1100AE50AE5057
:10024000AB98AB8811001B501C5C14E01C2AEACF51
:1002500007F0E9CF06F001EE00F01C50E926000E91
:10026000EA22EF50066E07C0EAFF06C0E9FFD88019
:10027000120004D0E868066ED8A0120012001B6AB3
:100280001C6A9D8A9F8AF28EF28C12009D9A01EE62
:1002900000F0010EF46EF36AF306000EF45AEE6AF3
:1002A000F450F310F9E11B6A1C6A9D8A1200F29E59
:1002B000E0CF9DFED8CF9EFEE8CF9FFEF28E0001DC
:1002C000A192B368E20EB26EF29E9DCEE0FF9ECE8A
:1002D000D8FF9FCEE8FFF28E10009EA8FED7AD6E2D
:1002E000120093948A94949A8B9A94988B989496EB
:1002F0008B9694948B9494928B9294908B90929AE8
:10030000899A9298899892968996929489949292D1
:10031000899292908990466A456A486A476A4A6A11
:10032000496A4C6A4B6A4E6A4D6A506A4F6A526A11
:10033000516A546A536A566A556A586A576A5A6AC1
:10034000596A5B6A5C6A5D6A5E6A5F6A606A616A72
:10035000626A636A646A656A286AFEEC0DF0E1EC21
:1003600011F000EC10F0010E1E6E800E1E5CD8B075
:10037000D0D102EE9DF0D8901E34E926000EEA227C
:10038000EECF04F0EFCF05F004C00DF005C00EF085
:10039000E5DE9A0E146E990E136E190E126E800E13
:1003A000116E3BDE88DE006E0EC001F002EE9DF0A5
:1003B000D8901E34E926000EEA2200C0EEFF01C0EC
:1003C000EFFF03EE9DF0D8901E34E926000EEA22DE
:1003D000EECF04F0EFCF05F004C00DF005C00EF035
:1003E000BDDE9A0E146E990E136E190E126E800EEB
:1003F000116E13DE60DE006E0EC001F003EE9DF0A4
:10040000D8901E34E926000EEA2200C0EEFF01C09B
:10041000EFFF04EE9DF0D8901E34E926000EEA228C
:10042000EECF04F0EFCF05F004C00DF005C00EF0E4
:1004300095DE9A0E146E990E136E190E126E800EC2
:10044000116E0DEC00F037DE006E0EC001F004EE10
:100450009DF0D8901E34E926000EEA2200C0EEFF7F
:1004600001C0EFFF05EE9DF0D8901E34E926000E86
:10047000EA22EECF04F0EFCF05F004C00DF005C086
:100480000EF06CDE9A0E146E990E136E190E126E2B
:10049000800E116E0DEC00F00EDE006E0EC001F04D
:1004A00005EE9DF0D8901E34E926000EEA2200C029
:1004B000EEFF01C0EFFF06EE9DF0D8901E34E92656
:1004C000000EEA22EECF04F0EFCF05F004C00DF0ED
:1004D00005C00EF043DE9A0E146E990E136E190EBF
:1004E000126E800E116E0DEC00F05BEC00F0006EF1
:1004F0000EC001F006EE9DF0D8901E34E926000EE5
:10050000EA2200C0EEFF01C0EFFF07EE9DF0D89099
:100510001E34E926000EEA22EECF04F0EFCF05F0FC
:1005200004C00DF005C00EF019DE9A0E146E990E7F
:10053000136E190E126E800E116E0DEC00F05BEC56
:1005400000F0006E0EC001F007EE9DF0D8901E3452
:10055000E926000EEA2200C0EEFF01C0EFFF08EE20
:100560009DF0D8901E34E926000EEA22EECF04F06A
:10057000EFCF05F004C00DF005C00EF0AEEC00F0BA
:100580009A0E146E990E136E190E126E800E116E65
:100590000DEC00F05BEC00F0006E0EC001F008EE18
:1005A0009DF0D8901E34E926000EEA2200C0EEFF2E
:1005B00001C0EFFF09EE9DF0D8901E34E926000E31
:1005C000EA22EECF04F0EFCF05F004C00DF005C035
:1005D0000EF0AEEC00F09A0E146E990E136E190E1A
:1005E000126E800E116E0DEC00F05BEC00F0006EF0
:1005F0000EC001F009EE9DF0D8901E34E926000EE1
:10060000EA2200C0EEFF01C0EFFF0AEE9DF0D89095
:100610001E34E926000EEA22EECF04F0EFCF05F0FB
:1006200004C00DF005C00EF0AEEC00F09A0E146E92
:10063000990E136E190E126E800E116E0DEC00F0F5
:100640005BEC00F0006E0EC001F00AEE9DF0D89059
:100650001E34E926000EEA2200C0EEFF01C0EFFFC3
:100660000BEE9DF0D8901E34E926000EEA22EECF64
:1006700004F0EFCF05F004C00DF005C00EF0AEECB5
:1006800000F09A0E146E990E136E190E126E800EF3
:10069000116E0DEC00F05BEC00F0006E0EC001F08E
:1006A0000BEE9DF0D8901E34E926000EEA2200C021
:1006B000EEFF01C0EFFF0CEE9DF0D8901E34E9264E
:1006C000000EEA22EECF04F0EFCF05F004C00DF0EB
:1006D00005C00EF0AEEC00F09A0E146E990E136E7B
:1006E000190E126E800E116E0DEC00F05BEC00F036
:1006F000006E0EC001F00CEE9DF0D8901E34E9267D
:10070000000EEA2200C0EEFF01C0EFFF1E2AD8A0B3
:100710002CD6276A266A256A246A936A8A6A3FEC7D
:1007200001F046EC01F0CD6AF294F28A870ED56EA4
:10073000B16AA19200EE6DF0300EEE68E82EFDD7A2
:100740006A68698E2C6A2B6A2A6A296A2D2AE86AE5
:100750002DB2010F2EB0010806E12E70292A000EDD
:100760002A222B222C2223EC01F01D6EBE0E1D5CD2
:1007700006E3FE0E1D5CD8A01F6AD2EF09F01DAE85
:1007800020D01F6A8D0E1D5C04E11DC01FF0206883
:1007900014D09D0E1D5C04E11DC01FF021680DD01A
:1007A000AD0E1D5C04E11DC01FF0236806D0BD0E18
:1007B0001D5C03E11DC01FF06B68D2EF09F0D0EFA4
:1007C00009F01F5204E1D2EF09F0D0EF09F08D0ECD
:1007D0001F5CD8A48BD0202805E11DC020F0D2EFEB
:1007E00009F082D0330E205C08E18B9A2490269089
:1007F00070686F686E686D6874D0390E205C03E0B5
:10080000450E205C08E124948B96269478687768DE
:100810007668756866D03C0E205C08E124968B945F
:1008200026967C687B687A6879685BD0410E205C8C
:1008300008E124988B92269880697F687E687D689D
:1008400050D0430E205C08E1249A8B90269A84694C
:1008500083698269816945D0440E205C08E1249C4B
:10086000899A269C88698769866985693AD0480E85
:10087000205C08E1249E8998269E8C698B698A6990
:1008800089692FD0550E205C08E125908996279024
:1008900090698F698E698D6924D0570E205C08E1BC
:1008A000259289942792946993699269916919D0E4
:1008B000580E205C08E125948992279498699769DD
:1008C000966995690ED0590E205C08E125968990AD
:1008D00027969C699B699A69996903D02068D2EF31
:1008E00009F02068D0EF09F0D0EF09F09D0E1F5CF1
:1008F000D8A4B7EF08F0212804E11DC021F0B6EF1D
:1009000008F01DC022F02252D8A482D0330E215C00
:1009100008E18B9A2490269070686F686E686D6805
:1009200074D0390E215C03E0450E215C08E124946B
:100930008B962694786877687668756866D03C0EE2
:10094000215C08E124968B9426967C687B687A6803
:1009500079685BD0410E215C08E124988B9226983F
:1009600080697F687E687D6850D0430E215C08E115
:10097000249A8B90269A846983698269816945D01B
:10098000440E215C08E1249C899A269C8869876929
:10099000866985693AD0480E215C08E1249E8998D1
:1009A000269E8C698B698A6989692FD0550E215CD6
:1009B00008E125908996279090698F698E698D69E5
:1009C00024D0570E215C08E12592899427929469DE
:1009D00093699269916919D0580E215C08E12594B8
:1009E0008992279498699769966995690ED0590EEE
:1009F000215C08E12596899027969C699B699A69F4
:100A0000996903D02168D2EF09F02168D0EF09F08D
:100A10002852D8B4B2EF08F0330E215CD8A451D0DC
:100A20008B8A02EE9DF0D8902234E926000EEA224D
:100A3000EECF2FF0EFCF30F024802F502924006E1E
:100A400030502A20016E000E2B20026E000E2C204A
:100A5000036E03C070F002C06FF001C06EF000C002
:100A60006DF05B522CE026800DEE9DF0D8905B344B
:100A7000E926000EEA22EECF00F0EFCF01F0D89089
:100A80002F34046E3034056E0050045C015005585C
:100A900005E330C046F02FC045F011D00DEE9DF0BB
:100AA000D8905B34E926000EEA22EECF00F0EFCFBB
:100AB00001F02F50005C456E30500158466EB1EF8A
:100AC00008F0390E215C04E0450E215CD8A451D019
:100AD0008B8603EE9DF0D8902234E926000EEA22A0
:100AE000EECF31F0EFCF32F0248431502924006E64
:100AF00032502A20016E000E2B20026E000E2C2098
:100B0000036E03C078F002C077F001C076F000C039
:100B100075F05C522CE026840DEE9DF0D8905C348C
:100B2000E926000EEA22EECF00F0EFCF01F0D890D8
:100B30003134046E3234056E0050045C01500558A7
:100B400005E332C048F031C047F011D00DEE9DF002
:100B5000D8905C34E926000EEA22EECF00F0EFCF09
:100B600001F03150005C476E32500158486EB1EFD1
:100B700008F03C0E215CD8A451D004EE9DF0D89032
:100B80002234E926000EEA22EECF33F0EFCF34F024
:100B90008B84248633502924006E34502A20016E21
:100BA000000E2B20026E000E2C20036E03C07CF082
:100BB00002C07BF001C07AF000C079F05D522CE0F9
:100BC00026860DEE9DF0D8905D34E926000EEA22CF
:100BD000EECF00F0EFCF01F0D8903334046E343410
:100BE000056E0050045C0150055805E334C04AF01E
:100BF00033C049F011D00DEE9DF0D8905D34E92658
:100C0000000EEA22EECF00F0EFCF01F03350005C8F
:100C1000496E345001584A6EB1EF08F0410E215C24
:100C2000D8A451D005EE9DF0D8902234E926000ECC
:100C3000EA22EECF35F0EFCF36F08B8224883550A4
:100C40002924006E36502A20016E000E2B20026EE1
:100C5000000E2C20036E03C080F002C07FF001C0A4
:100C60007EF000C07DF05E522CE026880DEE9DF0F7
:100C7000D8905E34E926000EEA22EECF00F0EFCFE6
:100C800001F0D8903534046E3634056E0050045CA3
:100C90000150055805E336C04CF035C04BF011D07B
:100CA0000DEE9DF0D8905E34E926000EEA22EECFDC
:100CB00000F0EFCF01F03550005C4B6E365001581C
:100CC0004C6EB1EF08F0430E215CD8A450D006EE74
:100CD0009DF0D8902234E926000EEA22EECF37F0BC
:100CE000EFCF38F08B80248A37502924006E38509B
:100CF0002A20016E000E2B20026E000E2C20036EA7
:100D000003C084F002C083F001C082F000C081F013
:100D10005F522CE0268A0DEE9DF0D8905F34E926D4
:100D2000000EEA22EECF00F0EFCF01F0D89037347A
:100D3000046E3834056E0050045C0150055805E31C
:100D400038C04EF037C04DF011D00DEE9DF0D89068
:100D50005F34E926000EEA22EECF00F0EFCF01F07B
:100D60003750005C4D6E385001584E6EFAD1440E2B
:100D7000215CD8A450D007EE9DF0D8902234E9260B
:100D8000000EEA22EECF39F0EFCF3AF0898A248CB8
:100D900039502924006E3A502A20016E000E2B2073
:100DA000026E000E2C20036E03C088F002C087F094
:100DB00001C086F000C085F060522CE0268C0DEE5C
:100DC0009DF0D8906034E926000EEA22EECF00F0C4
:100DD000EFCF01F0D8903934046E3A34056E0050EC
:100DE000045C0150055805E33AC050F039C04FF09B
:100DF00011D00DEE9DF0D8906034E926000EEA2265
:100E0000EECF00F0EFCF01F03950005C4F6E3A505A
:100E10000158506EA6D1480E215CD8A450D008EEDF
:100E20009DF0D8902234E926000EEA22EECF3BF066
:100E3000EFCF3CF08988248E3B502924006E3C5033
:100E40002A20016E000E2B20026E000E2C20036E55
:100E500003C08CF002C08BF001C08AF000C089F0A2
:100E600061522CE0268E0DEE9DF0D8906134E9267B
:100E7000000EEA22EECF00F0EFCF01F0D8903B3425
:100E8000046E3C34056E0050045C0150055805E3C7
:100E90003CC052F03BC051F011D00DEE9DF0D89007
:100EA0006134E926000EEA22EECF00F0EFCF01F028
:100EB0003B50005C516E3C500158526E52D1550E61
:100EC000215CD8A450D009EE9DF0D8902234E926B8
:100ED000000EEA22EECF3DF0EFCF3EF0898625806E
:100EE0003D502924006E3E502A20016E000E2B201A
:100EF000026E000E2C20036E03C090F002C08FF033
:100F000001C08EF000C08DF062522CE027800DEE03
:100F10009DF0D8906234E926000EEA22EECF00F070
:100F2000EFCF01F0D8903D34046E3E34056E005092
:100F3000045C0150055805E33EC054F03DC053F039
:100F400011D00DEE9DF0D8906234E926000EEA2211
:100F5000EECF00F0EFCF01F03D50005C536E3E50FD
:100F60000158546EFED0570E215CD8A450D00AEE22
:100F70009DF0D8902234E926000EEA22EECF3FF011
:100F8000EFCF40F0898425823F502924006E4050E5
:100F90002A20016E000E2B20026E000E2C20036E04
:100FA00003C094F002C093F001C092F000C091F031
:100FB00063522CE027820DEE9DF0D8906334E92631
:100FC000000EEA22EECF00F0EFCF01F0D8903F34D0
:100FD000046E4034056E0050045C0150055805E372
:100FE00040C056F03FC055F011D00DEE9DF0D890A6
:100FF0006334E926000EEA22EECF00F0EFCF01F0D5
:101000003F50005C556E40500158566EAAD0580EA5
:10101000215CD8A450D00BEE9DF0D8902234E92664
:10102000000EEA22EECF41F0EFCF42F08982258414
:1010300041502924006E42502A20016E000E2B20C0
:10104000026E000E2C20036E03C098F002C097F0D1
:1010500001C096F000C095F064522CE027840DEE9C
:101060009DF0D8906434E926000EEA22EECF00F01D
:10107000EFCF01F0D8904134046E4234056E005039
:10108000045C0150055805E342C058F041C057F0D8
:1010900011D00DEE9DF0D8906434E926000EEA22BE
:1010A000EECF00F0EFCF01F04150005C576E4250A0
:1010B0000158586E56D0590E215CD8A450D00CEE71
:1010C0009DF0D8902234E926000EEA22EECF43F0BC
:1010D000EFCF44F08980258643502924006E445088
:1010E0002A20016E000E2B20026E000E2C20036EB3
:1010F00003C09CF002C09BF001C09AF000C099F0C0
:1011000065522CE027860DEE9DF0D8906534E926D7
:10111000000EEA22EECF00F0EFCF01F0D89043347A
:10112000046E4434056E0050045C0150055805E31C
:1011300044C05AF043C059F011D00DEE9DF0D89044
:101140006534E926000EEA22EECF00F0EFCF01F081
:101150004350005C596E445001585A6E02D02168C9
:1011600021D102D021681ED121681AD119D1AD0E2A
:101170001F5CD8A408D1232804E11DC023F012D19C
:1011800001D1330E235C14E11DC05BF05B520CE017
:101190000DEE9DF0D8905B34E926000EEA22EECFEA
:1011A00045F0EFCF46F003D0466A456A2690E8D076
:1011B000390E235C03E0450E235C14E11DC05CF096
:1011C0005C520CE00DEE9DF0D8905C34E926000EE8
:1011D000EA22EECF47F0EFCF48F003D0486A476AE3
:1011E0002694CED03C0E235C14E11DC05DF05D5210
:1011F0000CE00DEE9DF0D8905D34E926000EEA2259
:10120000EECF49F0EFCF4AF003D04A6A496A2696FA
:10121000B7D0410E235C14E11DC05EF05E520CE0BD
:101220000DEE9DF0D8905E34E926000EEA22EECF56
:101230004BF0EFCF4CF003D04C6A4B6A2698A0D00D
:10124000430E235C14E11DC05FF05F520CE00DEE15
:101250009DF0D8905F34E926000EEA22EECF4DF0E3
:10126000EFCF4EF003D04E6A4D6A269A89D0440ED5
:10127000235C14E11DC060F060520CE00DEE9DF0A7
:10128000D8906034E926000EEA22EECF4FF0EFCF7F
:1012900050F003D0506A4F6A269C72D0480E235CEF
:1012A00014E11DC061F061520CE00DEE9DF0D8908C
:1012B0006134E926000EEA22EECF51F0EFCF52F072
:1012C00003D0526A516A269E5BD0550E235C14E10E
:1012D0001DC062F062520CE00DEE9DF0D8906234B9
:1012E000E926000EEA22EECF53F0EFCF54F003D000
:1012F000546A536A279044D0570E235C14E11DC0F2
:1013000063F063520CE00DEE9DF0D8906334E92653
:10131000000EEA22EECF55F0EFCF56F003D0566A1A
:10132000556A27922DD0580E235C14E11DC064F03D
:1013300064520CE00DEE9DF0D8906434E926000E66
:10134000EA22EECF57F0EFCF58F003D0586A576A31
:10135000279416D0590E235C13E11DC065F0655229
:101360000CE00DEE9DF0D8906534E926000EEA22DF
:10137000EECF59F0EFCF5AF003D05A6A596A279648
:10138000236810D00DD0BD0E1F5C0AE16B2804E16C
:101390001DC06BF007D004D01DC06CF0D8EC0CF071
:1013A0009EEC0CF00C0E6A5CD8B095EF0CF0665019
:1013B000295C67502A5868502B5869502C58D8A07F
:1013C00078EF0CF0698E6A523AE126B007D024908B
:1013D0008B9A70686F686E686D682FD024A017D0E4
:1013E0008B9A45502924006E46502A20016E000E2B
:1013F0002B20026E000E2C20036E03C070F002C082
:101400006FF001C06EF000C06DF0249016D08B8A92
:101410002F502924006E30502A20016E000E2B2000
:10142000026E000E2C20036E03C070F002C06FF03D
:1014300001C06EF000C06DF0248077EF0CF0020E5A
:101440006A5C3AE126B407D024948B967868776872
:10145000766875682FD024A417D08B96475029241E
:10146000006E48502A20016E000E2B20026E000EE6
:101470002C20036E03C078F002C077F001C076F034
:1014800000C075F0249416D08B8631502924006E4C
:1014900032502A20016E000E2B20026E000E2C20EE
:1014A000036E03C078F002C077F001C076F000C090
:1014B00075F0248477EF0CF0030E6A5C39E126B6F0
:1014C00007D024968B947C687B687A6879682FD0E3
:1014D00024A617D08B9449502924006E4A502A2004
:1014E000016E000E2B20026E000E2C20036E03C036
:1014F0007CF002C07BF001C07AF000C079F0249645
:1015000016D08B8433502924006E34502A20016E6B
:10151000000E2B20026E000E2C20036E03C07CF008
:1015200002C07BF001C07AF000C079F02486DFD1E0
:10153000040E6A5C39E126B807D024988B92806942
:101540007F687E687D682FD024A817D08B924B507F
:101550002924006E4C502A20016E000E2B20026EB2
:10156000000E2C20036E03C080F002C07FF001C08B
:101570007EF000C07DF0249816D08B82355029244F
:10158000006E36502A20016E000E2B20026E000ED7
:101590002C20036E03C080F002C07FF001C07EF0FB
:1015A00000C07DF02488A3D1050E6A5C39E126BA1B
:1015B00007D0249A8B9084698369826981692FD0CE
:1015C00024AA17D08B904D502924006E4E502A200B
:1015D000016E000E2B20026E000E2C20036E03C045
:1015E00084F002C083F001C082F000C081F0249A30
:1015F00016D08B8037502924006E38502A20016E77
:10160000000E2B20026E000E2C20036E03C084F00F
:1016100002C083F001C082F000C081F0248A67D14B
:10162000060E6A5C39E126BC07D0249C899A886939
:101630008769866985692FD024AC17D0899A4F5065
:101640002924006E50502A20016E000E2B20026EBD
:10165000000E2C20036E03C088F002C087F001C08A
:1016600086F000C085F0249C16D0898A3950292440
:10167000006E3A502A20016E000E2B20026E000EE2
:101680002C20036E03C088F002C087F001C086F0F2
:1016900000C085F0248C2BD1070E6A5C39E126BE90
:1016A00007D0249E89988C698B698A6989692FD0B3
:1016B00024AE17D0899851502924006E52502A2008
:1016C000016E000E2B20026E000E2C20036E03C054
:1016D0008CF002C08BF001C08AF000C089F0249E1B
:1016E00016D089883B502924006E3C502A20016E78
:1016F000000E2B20026E000E2C20036E03C08CF017
:1017000002C08BF001C08AF000C089F0248EEFD0B7
:10171000080E6A5C39E127B007D025908996906958
:101720008F698E698D692FD025A017D08996535067
:101730002924006E54502A20016E000E2B20026EC8
:10174000000E2C20036E03C090F002C08FF001C089
:101750008EF000C08DF0259016D089863D5029244A
:10176000006E3E502A20016E000E2B20026E000EED
:101770002C20036E03C090F002C08FF001C08EF0E9
:1017800000C08DF02580B3D0090E6A5C39E127B224
:1017900007D02592899494699369926991692FD0B1
:1017A00025A217D0899455502924006E56502A201E
:1017B000016E000E2B20026E000E2C20036E03C063
:1017C00094F002C093F001C092F000C091F0259215
:1017D00016D089843F502924006E40502A20016E83
:1017E000000E2B20026E000E2C20036E03C094F01E
:1017F00002C093F001C092F000C091F0258277D032
:101800000A0E6A5C39E127B407D025948992986959
:101810009769966995692FD025A417D0899257505A
:101820002924006E58502A20016E000E2B20026ED3
:10183000000E2C20036E03C098F002C097F001C088
:1018400096F000C095F0259416D089824150292445
:10185000006E42502A20016E000E2B20026E000EF8
:101860002C20036E03C098F002C097F001C096F0E0
:1018700000C095F025843BD00B0E6A5C38E127B69A
:1018800007D0259689909C699B699A6999692FD0A0
:1018900025A617D0899059502924006E5A502A2025
:1018A000016E000E2B20026E000E2C20036E03C072
:1018B0009CF002C09BF001C09AF000C099F0259600
:1018C00016D0898043502924006E44502A20016E8E
:1018D000000E2B20026E000E2C20036E03C09CF025
:1018E00002C09BF001C09AF000C099F0258626D86E
:1018F0002CAE1AD02C6A2B6A2A6A296A256A246AB5
:10190000276A266A00EE6DF0300EEE68E82EFDD7ED
:101910008B9A8B988B968B948B928B90899A8998C3
:10192000899689948992899006D02CAE04D02C6A2D
:101930002B6A2A6A296A8170A6EF03F06A68698EA9
:101940001E6A0C0E1E5C33E2D8901E34E96EEA6A01
:10195000EA36E936EA366D0EE926000EEA22EFCFC6
:1019600000F0ECCF01F0ECCF02F0ECCF03F06650CA
:10197000005C67500158685002586950035815E2DE
:10198000D8901E34E96EEA6AEA36E936EA366D0E18
:10199000E926000EEA22EFCF66F0ECCF67F0ECCF3D
:1019A00068F0ECCF69F01EC06AF01E2ACAE312008C
:1019B0001E0E6B5CD8A4B6D06C5224E1276A266A4E
:1019C000466A456A5B6A486A476A5C6A4A6A496A63
:1019D0005D6A4C6A4B6A5E6A4E6A4D6A5F6A506A1B
:1019E0004F6A606A526A516A616A546A536A626AEB
:1019F000566A556A636A586A576A646A5A6A596AC3
:101A0000656A8FD06CC05BF00DEE9DF0D8906C34A1
:101A1000E926000EEA22EECF45F0EFCF46F06CC08B
:101A20005CF00DEE9DF0D8906C34E926000EEA22B1
:101A3000EECF47F0EFCF48F06CC05DF00DEE9DF0BB
:101A4000D8906C34E926000EEA22EECF49F0EFCFB1
:101A50004AF06CC05EF00DEE9DF0D8906C34E92633
:101A6000000EEA22EECF4BF0EFCF4CF06CC05FF0EF
:101A70000DEE9DF0D8906C34E926000EEA22EECFF0
:101A80004DF0EFCF4EF06CC060F00DEE9DF0D890B1
:101A90006C34E926000EEA22EECF4FF0EFCF50F083
:101AA0006CC061F00DEE9DF0D8906C34E926000E0C
:101AB000EA22EECF51F0EFCF52F06CC062F00DEEA3
:101AC0009DF0D8906C34E926000EEA22EECF53F058
:101AD000EFCF54F06CC063F00DEE9DF0D8906C34F5
:101AE000E926000EEA22EECF55F0EFCF56F06CC09B
:101AF00064F00DEE9DF0D8906C34E926000EEA22D9
:101B0000EECF57F0EFCF58F06CC065F00DEE9DF0C2
:101B1000D8906C34E926000EEA22EECF59F0EFCFD0
:101B20005AF06AD0420E6B5CD8A448D06C52D8A44C
:101B30003FD0256A246A276A266A00EE6DF0300ECF
:101B4000EE68E82EFDD76A688B9A8B988B968B94FB
:101B50008B928B90899A8998899689948992899099
:101B6000466A456A486A476A4A6A496A4C6A4B6AE1
:101B70004E6A4D6A506A4F6A526A516A546A536A91
:101B8000566A556A586A576A5A6A596A5B6A5C6A41
:101B90005D6A5E6A5F6A606A616A626A636A646AF1
:101BA000656A286A8A942C6A2B6A2A6A296A05D08F
:101BB000285203E18A846CC028F01ED07B0E6B5C37
:101BC0001BE1256A246A276A266A8B9A8B988B9672
:101BD0008B948B928B90899A899889968994899213
:101BE00089902C6A2B6A2A6A296A00EE6DF0300E01
:101BF000EE68E82EFDD76A686B6812000D019E69D9
:101C00009D69A20EA06FC30E9F6F9A0EA26F460E23
:101C1000A16F960EA46F320EA36F920EA66F3A0EAE
:101C2000A56F8E0EA86F5D0EA76F8A0EAA6F9A0E13
:101C3000A96F860EAC6FF00EAB6F830EAE6F5F0EAA
:101C4000AD6F7F0EB06FE70EAF6F7C0EB26F850E7B
:101C5000B16F790EB46F3B0EB36F760EB66F070E91
:101C6000B56F720EB86FE80EB76F6F0EBA6FDF0EFA
:101C7000B96F6C0EBC6FEA0EBB6F6A0EBE6F0A0EB8
:101C8000BD6F670EC06F3C0EBF6F640EC26F820ED9
:101C9000C16F610EC46FDA0EC36F5F0EC66F440E64
:101CA000C56F5C0EC86FBF0EC76F5A0ECA6F4C0E61
:101CB000C96F570ECC6FE90ECB6F550ECE6F960ED7
:101CC000CD6F530ED06FCF6F510ED26F200ED16FEC
:101CD0004E0ED46FFB0ED36F4C0ED66FE50ED56F44
:101CE0004A0ED86FDC0ED76F480EDA6FE20ED96F4E
:101CF000460EDC6FF50EDB6F450EDE6F150EDD6FE9
:101D0000430EE06F420EDF6F410EE26F7B0EE16F1C
:101D10003F0EE46FC00EE36F3E0EE66F100EE56FF0
:101D20003C0EE86F6D0EE76F3A0EEA6FD40EE96F66
:101D3000390EEC6F460EEB6F370EEE6FC20EED6F85
:101D4000360EF06F490EEF6F340EF26FDA0EF16F50
:101D5000330EF46F740EF36F320EF66F180EF56FCC
:101D6000300EF86FC50EF76F2F0EFA6F7B0EF96FFE
:101D70002E0EFC6F3A0EFB6F2D0EFE6F020EFD6FE6
:101D80002B0E0E01006FD10E0D01FF6F2A0E0E01FA
:101D9000026FA90E016F290E046F880E036F280EC3
:101DA000066F6F0E056F270E086F5E0E076F260E0B
:101DB0000A6F530E096F250E0C6F500E0B6F240E19
:101DC0000E6F540E0D6F230E106F5E0E0F6F220EEE
:101DD000126F6F0E116F210E146F860E136F200E8F
:101DE000166FA30E156F1F0E186FC60E176F1E0EFF
:101DF0001A6FEF0E196F1E0E1C6F1B6F1D0E1E6FDC
:101E0000520E1D6F1C0E206F8C0E1F6F1B0E226F4B
:101E1000CB0E216F1B0E246F0F0E236F1A0E266F31
:101E2000580E256F190E286FA50E276F180E2A6FF2
:101E3000F80E296F180E2C6F4F0E2B6F170E2E6F8A
:101E4000AB0E2D6F170E306F0A0E2F6F160E326FFE
:101E50006F0E316F150E346FD70E336F150E366F50
:101E6000430E356F140E386FB30E376F140E3A6F82
:101E7000270E396F130E3C6F9F0E3B6F130E3E6F94
:101E80001A0E3D6F120E406F990E3F6F120E426F89
:101E90001B0E416F110E446FA10E436F110E466F62
:101EA000290E456F100E486FB50E476F100E4A6F22
:101EB000440E496F0F0E4C6FD60E4B6F0F0E4E6FC8
:101EC0006B0E4D6F0F0E506F030E4F6F0E0E526F55
:101ED0009D0E516F0E0E546F3A0E536F0D0E566FCE
:101EE000DA0E556F0D0E586F7C0E576F0D0E5A6F30
:101EF000210E596F0C0E5C6FC80E5B6F0C0E5E6F7F
:101F0000720E5D6F0C0E606F1E0E5F6F0B0E626FB8
:101F1000CC0E616F0B0E646F7C0E636F0B0E666FE1
:101F20002E0E656F0A0E686FE30E676F0A0E6A6FFA
:101F3000990E696F0A0E6C6F510E6B6F0A0E6E6F01
:101F40000B0E6D6F090E706FC80E6F6F090E726FFA
:101F5000850E716F090E746F450E736F090E766FE3
:101F6000060E756F080E786FC90E776F080E7A6FC0
:101F70008E0E796F080E7C6F540E7B6F080E7E6F8D
:101F80001C0E7D6F070E806FE50E7F6F070E826F50
:101F9000AF0E816F070E846F7B0E836F070E866F07
:101FA000490E856F070E886F170E876F060E8A6FB2
:101FB000E70E896F060E8C6FB90E8B6F060E8E6F53
:101FC0008B0E8D6F060E906F5F0E8F6F060E926FE9
:101FD000340E916F060E946F0A0E936F050E966F76
:101FE000E10E956F050E986FB90E976F050E9A6FFB
:101FF000930E996F050E9C6F6D0E9B6F0001120082
:102000000201A06B7E0E9F6FA26B820EA16FA46B6C
:10201000860EA36FA66B8A0EA56FA86B8F0EA76F97
:10202000AA6B930EA96FAC6B970EAB6FAE6B9B0E4A
:10203000AD6FB06BA00EAF6FB26BA40EB16FB46B8F
:10204000A80EB36FB66BAC0EB56FB86BB10EB76FB1
:10205000BA6BB50EB96FBC6BB90EBB6FBE6BBD0E64
:10206000BD6FC06BC20EBF6FC26BC60EC16FC46BBB
:10207000CA0EC36FC66BCE0EC56FC86BD30EC76FCB
:10208000CA6BD70EC96FCC6BDB0ECB6FCE6BDF0E7E
:10209000CD6FD06BE40ECF6FD26BE80ED16FD46BE7
:1020A000EC0ED36FD66BF00ED56FD86BF50ED76FE5
:1020B000DA6BF90ED96FDC6BFD0EDB6F010EDE6F94
:1020C000DD6FE06F060EDF6F010EE26F0A0EE16F4B
:1020D000010EE46F0E0EE36F010EE66F120EE56F58
:1020E000010EE86F170EE76F010EEA6F1B0EE96F26
:1020F000010EEC6F1F0EEB6F010EEE6F230EED6FF6
:10210000010EF06F280EEF6F010EF26F2C0EF16FC3
:10211000010EF46F300EF36F010EF66F350EF56F92
:10212000010EF86F390EF76F010EFA6F3D0EF96F61
:10213000010EFC6F410EFB6F010EFE6F460EFD6F30
:10214000010E0301006F4A0E0201FF6F010E030131
:10215000026F4E0E016F010E046F520E036F010EDF
:10216000066F570E056F010E086F5B0E076F010EAD
:102170000A6F5F0E096F010E0C6F630E0B6F010E7D
:102180000E6F680E0D6F010E106F6C0E0F6F010E4B
:10219000126F700E116F010E146F740E136F010E1B
:1021A000166F790E156F010E186F7D0E176F010EE9
:1021B0001A6F810E196F010E1C6F850E1B6F010EB9
:1021C0001E6F8A0E1D6F010E206F8E0E1F6F010E87
:1021D000226F920E216F010E246F960E236F010E57
:1021E000266F9B0E256F010E286F9F0E276F010E25
:1021F0002A6FA30E296F010E2C6FA70E2B6F010EF5
:102200002E6FAC0E2D6F010E306FB00E2F6F010EC2
:10221000326FB40E316F010E346FB80E336F010E92
:10222000366FBD0E356F010E386FC10E376F010E60
:102230003A6FC50E396F010E3C6FC90E3B6F010E30
:102240003E6FCE0E3D6F010E406FD20E3F6F010EFE
:10225000426FD60E416F010E446FDA0E436F010ECE
:10226000466FDF0E456F010E486FE30E476F010E9C
:102270004A6FE70E496F010E4C6FEC0E4B6F010E6B
:102280004E6FF00E4D6F010E506FF40E4F6F010E3A
:10229000526FF80E516F010E546FFD0E536F020E08
:1022A000566F010E556F020E586F050E576F020ED6
:1022B0005A6F090E596F020E5C6F0E0E5B6F020EA5
:1022C0005E6F120E5D6F020E606F160E5F6F020E74
:1022D000626F1A0E616F020E646F1F0E636F020E43
:1022E000666F230E656F020E686F270E676F020E12
:1022F0006A6F2B0E696F020E6C6F300E6B6F020EE1
:102300006E6F340E6D6F020E706F380E6F6F020EAF
:10231000726F3C0E716F020E746F410E736F020E7E
:10232000766F450E756F020E786F490E776F020E4D
:102330007A6F4D0E796F020E7C6F520E7B6F020E1C
:102340007E6F560E7D6F020E806F5A0E7F6F020EEB
:10235000826F5E0E816F020E846F630E836F020EBA
:10236000866F670E856F020E886F6B0E876F020E89
:102370008A6F6F0E896F020E8C6F740E8B6F020E58
:102380008E6F780E8D6F020E906F7C0E8F6F020E27
:10239000926F800E916F020E946F850E936F020EF6
:1023A000966F890E956F020E986F8D0E976F020EC5
:1023B0009A6F910E996F020E9C6F960E9B6F0001A3
:1023C00012000401A06B8C0E9F6FA26B8E0EA16F8A
:1023D000A46B900EA36FA66B910EA56FA86B930EC6
:1023E000A76FAA6B950EA96FAC6B960EAB6FAE6B19
:1023F000980EAD6FB06B9A0EAF6FB26B9C0EB16F53
:10240000B46B9D0EB36FB66B9F0EB56FB86BA10E1C
:10241000B76FBA6BA20EB96FBC6BA40EBB6FBE6B6D
:10242000A60EBD6FC06BA80EBF6FC26BA90EC16FA9
:10243000C46BAB0EC36FC66BAD0EC56FC86BAE0E73
:10244000C76FCA6BB00EC96FCC6BB20ECB6FCE6BC1
:10245000B30ECD6FD06BB50ECF6FD26BB70ED16F01
:10246000D46BB90ED36FD66BBA0ED56FD86BBC0ECA
:10247000D76FDA6BBE0ED96FDC6BBF0EDB6FDE6B16
:10248000C10EDD6FE06BC30EDF6FE26BC40EE16F58
:10249000E46BC60EE36FE66BC80EE56FE86BCA0E21
:1024A000E76FEA6BCB0EE96FEC6BCD0EEB6FEE6B6B
:1024B000CF0EED6FF06BD00EEF6FF26BD20EF16FAF
:1024C000F46BD40EF36FF66BD50EF56FF86BD70E79
:1024D000F76FFA6BD90EF96FFC6BDB0EFB6FFE6BBF
:1024E000DC0EFD6F0501006BDE0E0401FF6F0501C0
:1024F000026BE00E016F046BE10E036F066BE30EDF
:10250000056F086BE50E076F0A6BE60E096F0C6B23
:10251000E80E0B6F0E6BEA0E0D6F106BEC0E0F6F6B
:10252000126BED0E116F146BEF0E136F166BF10E35
:10253000156F186BF20E176F1A6BF40E196F1C6B78
:10254000F60E1B6F1E6BF80E1D6F206BF90E1F6FC2
:10255000226BFB0E216F246BFD0E236F266BFE0E8C
:10256000256F010E286F276B2A6F020E296F010E4F
:102570002C6F030E2B6F010E2E6F050E2D6F010EAB
:10258000306F070E2F6F010E326F090E316F010E83
:10259000346F0A0E336F010E366F0C0E356F010E5D
:1025A000386F0E0E376F010E3A6F0F0E396F010E36
:1025B0003C6F110E3B6F010E3E6F130E3D6F010E0F
:1025C000406F140E3F6F010E426F160E416F010EE9
:1025D000446F180E436F010E466F1A0E456F010EC1
:1025E000486F1B0E476F010E4A6F1D0E496F010E9B
:1025F0004C6F1F0E4B6F010E4E6F200E4D6F010E74
:10260000506F220E4F6F010E526F240E516F010E4C
:10261000546F250E536F010E566F270E556F010E26
:10262000586F290E576F010E5A6F2B0E596F010EFE
:102630005C6F2C0E5B6F010E5E6F2E0E5D6F010ED8
:10264000606F300E5F6F010E626F310E616F010EB1
:10265000646F330E636F010E666F350E656F010E8A
:10266000686F360E676F010E6A6F380E696F010E64
:102670006C6F3A0E6B6F010E6E6F3C0E6D6F010E3C
:10268000706F3D0E6F6F010E726F3F0E716F010E16
:10269000746F410E736F010E766F420E756F010EEF
:1026A000786F440E776F010E7A6F460E796F010EC8
:1026B0007C6F480E7B6F010E7E6F490E7D6F010EA1
:1026C000806F4B0E7F6F010E826F4D0E816F010E7A
:1026D000846F4E0E836F010E866F500E856F010E54
:1026E000886F520E876F010E8A6F530E896F010E2D
:1026F0008C6F550E8B6F010E8E6F570E8D6F010E06
:10270000906F590E8F6F010E926F5A0E916F010EDE
:10271000946F5C0E936F010E966F5E0E956F010EB7
:10272000986F5F0E976F010E9A6F610E996F010E91
:102730009C6F630E9B6FA06BEF0E9F6FA26BF20EF0
:10274000A16FA46BF50EA36FA66BF90EA56FA86B16
:10275000FC0EA76FAA6BA969010EAC6F030EAB6FDD
:10276000010EAE6F060EAD6F010EB06F090EAF6FAA
:10277000010EB26F0D0EB16F010EB46F100EB36F7C
:10278000010EB66F140EB56F010EB86F170EB76F4E
:10279000010EBA6F1A0EB96F010EBC6F1E0EBB6F21
:1027A000010EBE6F210EBD6F010EC06F240EBF6FF4
:1027B000010EC26F280EC16F010EC46F2B0EC36FC6
:1027C000010EC66F2E0EC56F010EC86F320EC76F99
:1027D000010ECA6F350EC96F010ECC6F390ECB6F6B
:1027E000010ECE6F3C0ECD6F010ED06F3F0ECF6F3E
:1027F000010ED26F430ED16F010ED46F460ED36F10
:10280000010ED66F490ED56F010ED86F4D0ED76FE2
:10281000010EDA6F500ED96F010EDC6F540EDB6FB4
:10282000010EDE6F570EDD6F010EE06F5A0EDF6F87
:10283000010EE26F5E0EE16F010EE46F610EE36F59
:10284000010EE66F640EE56F010EE86F680EE76F2C
:10285000010EEA6F6B0EE96F010EEC6F6E0EEB6FFF
:10286000010EEE6F720EED6F010EF06F750EEF6FD1
:10287000010EF26F790EF16F010EF46F7C0EF36FA3
:10288000010EF66F7F0EF56F010EF86F830EF76F76
:10289000010EFA6F860EF96F010EFC6F890EFB6F49
:1028A000010EFE6F8D0EFD6F010E0601006F900E82
:1028B0000501FF6F010E0601026F930E016F010EFD
:1028C000046F970E036F010E066F9A0E056F010ECF
:1028D000086F9E0E076F010E0A6FA10E096F010EA1
:1028E0000C6FA40E0B6F010E0E6FA80E0D6F010E74
:1028F000106FAB0E0F6F010E126FAE0E116F010E47
:10290000146FB20E136F010E166FB50E156F010E18
:10291000186FB80E176F010E1A6FBC0E196F010EEB
:102920001C6FBF0E1B6F010E1E6FC30E1D6F010EBD
:10293000206FC60E1F6F010E226FC90E216F010E90
:10294000246FCD0E236F010E266FD00E256F010E62
:10295000286FD30E276F010E2A6FD70E296F010E35
:102960002C6FDA0E2B6F010E2E6FDE0E2D6F010E07
:10297000306FE10E2F6F010E326FE40E316F010EDA
:10298000346FE80E336F010E366FEB0E356F010EAC
:10299000386FEE0E376F010E3A6FF20E396F010E7F
:1029A0003C6FF50E3B6F010E3E6FF80E3D6F010E52
:1029B000406FFC0E3F6F010E426F4169020E446F83
:1029C000030E436F020E466F060E456F020E486FF0
:1029D000090E476F020E4A6F0D0E496F020E4C6FC3
:1029E000100E4B6F020E4E6F130E4D6F020E506F96
:1029F000170E4F6F020E526F1A0E516F020E546F68
:102A00001D0E536F020E566F210E556F020E586F3A
:102A1000240E576F020E5A6F280E596F020E5C6F0C
:102A20002B0E5B6F020E5E6F2E0E5D6F020E606FDF
:102A3000320E5F6F020E626F350E616F020E646FB1
:102A4000380E636F020E666F3C0E656F020E686F84
:102A50003F0E676F020E6A6F420E696F020E6C6F57
:102A6000460E6B6F020E6E6F490E6D6F020E706F29
:102A70004D0E6F6F020E726F500E716F020E746FFB
:102A8000530E736F020E766F570E756F020E786FCE
:102A90005A0E776F020E7A6F5D0E796F020E7C6FA1
:102AA000610E7B6F020E7E6F640E7D6F020E806F73
:102AB000680E7F6F020E826F6B0E816F020E846F45
:102AC0006E0E836F020E866F720E856F020E886F18
:102AD000750E876F020E8A6F780E896F020E8C6FEB
:102AE0007C0E8B6F020E8E6F7F0E8D6F020E906FBD
:102AF000820E8F6F020E926F860E916F020E946F90
:102B0000890E936F020E966F8D0E956F020E986F61
:102B1000900E976F020E9A6F930E996F020E9C6F34
:102B2000970E9B6FA06B910E9F6FA26B950EA16F7E
:102B3000A46B990EA36FA66B9D0EA56FA86BA20E3A
:102B4000A76FAA6BA60EA96FAC6BAA0EAB6FAE6B8C
:102B5000AE0EAD6FB06BB20EAF6FB26BB60EB16FA3
:102B6000B46BBA0EB36FB66BBE0EB56FB86BC20E58
:102B7000B76FBA6BC60EB96FBC6BCB0EBB6FBE6BBB
:102B8000CF0EBD6FC06BD30EBF6FC26BD70EC16FC0
:102B9000C46BDB0EC36FC66BDF0EC56FC86BE30E75
:102BA000C76FCA6BE70EC96FCC6BEB0ECB6FCE6BEA
:102BB000F00ECD6FD06BF40ECF6FD26BF80ED16FDD
:102BC000D46BFC0ED36F010ED66FD56BD86F040E8D
:102BD000D76F010EDA6F080ED96F010EDC6F0C0E85
:102BE000DB6F010EDE6F100EDD6F010EE06F140E55
:102BF000DF6F010EE26F190EE16F010EE46F1D0E23
:102C0000E36F010EE66F210EE56F010EE86F250EF2
:102C1000E76F010EEA6F290EE96F010EEC6F2D0EC2
:102C2000EB6F010EEE6F310EED6F010EF06F350E92
:102C3000EF6F010EF26F390EF16F010EF46F3D0E62
:102C4000F36F010EF66F420EF56F010EF86F460E30
:102C5000F76F010EFA6F4A0EF96F010EFC6F4E0E00
:102C6000FB6F010EFE6F520EFD6F010E0701006F2C
:102C7000560E0601FF6F010E0701026F5A0E016F1B
:102C8000010E046F5E0E036F010E066F620E056F7C
:102C9000010E086F660E076F010E0A6F6B0E096F4B
:102CA000010E0C6F6F0E0B6F010E0E6F730E0D6F1A
:102CB000010E106F770E0F6F010E126F7B0E116FEA
:102CC000010E146F7F0E136F010E166F830E156FBA
:102CD000010E186F870E176F010E1A6F8B0E196F8A
:102CE000010E1C6F8F0E1B6F010E1E6F940E1D6F59
:102CF000010E206F980E1F6F010E226F9C0E216F28
:102D0000010E246FA00E236F010E266FA40E256FF7
:102D1000010E286FA80E276F010E2A6FAC0E296FC7
:102D2000010E2C6FB00E2B6F010E2E6FB40E2D6F97
:102D3000010E306FB80E2F6F010E326FBD0E316F66
:102D4000010E346FC10E336F010E366FC50E356F35
:102D5000010E386FC90E376F010E3A6FCD0E396F05
:102D6000010E3C6FD10E3B6F010E3E6FD50E3D6FD5
:102D7000010E406FD90E3F6F010E426FDD0E416FA5
:102D8000010E446FE10E436F010E466FE60E456F74
:102D9000010E486FEA0E476F010E4A6FEE0E496F43
:102DA000010E4C6FF20E4B6F010E4E6FF60E4D6F13
:102DB000010E506FFA0E4F6F010E526FFE0E516FE3
:102DC000020E546F536F566F060E556F020E586FFA
:102DD0000A0E576F020E5A6F0F0E596F020E5C6F7C
:102DE000130E5B6F020E5E6F170E5D6F020E606F4B
:102DF0001B0E5F6F020E626F1F0E616F020E646F1B
:102E0000230E636F020E666F270E656F020E686FEA
:102E10002B0E676F020E6A6F2F0E696F020E6C6FBA
:102E2000330E6B6F020E6E6F380E6D6F020E706F89
:102E30003C0E6F6F020E726F400E716F020E746F58
:102E4000440E736F020E766F480E756F020E786F28
:102E50004C0E776F020E7A6F500E796F020E7C6FF8
:102E6000540E7B6F020E7E6F580E7D6F020E806FC8
:102E70005C0E7F6F020E826F610E816F020E846F97
:102E8000650E836F020E866F690E856F020E886F66
:102E90006D0E876F020E8A6F710E896F020E8C6F36
:102EA000750E8B6F020E8E6F790E8D6F020E906F06
:102EB0007D0E8F6F020E926F810E916F020E946FD6
:102EC000850E936F020E966F8A0E956F020E986FA5
:102ED0008E0E976F020E9A6F920E996F020E9C6F74
:102EE000960E9B6FA06B820E9F6FA26B840EA16FDC
:102EF000A46B860EA36FA66B880EA56FA86B8A0EB7
:102F0000A76FAA6B8B0EA96FAC6B8D0EAB6FAE6B00
:102F10008F0EAD6FB06B910EAF6FB26B920EB16F43
:102F2000B46B940EB36FB66B960EB56FB86B980E0C
:102F3000B76FBA6B9A0EB96FBC6B9B0EBB6FBE6B53
:102F40009D0EBD6FC06B9F0EBF6FC26BA10EC16F98
:102F5000C46BA20EC36FC66BA40EC56FC86BA60E62
:102F6000C76FCA6BA80EC96FCC6BAA0ECB6FCE6BA6
:102F7000AB0ECD6FD06BAD0ECF6FD26BAF0ED16FEE
:102F8000D46BB10ED36FD66BB20ED56FD86BB40EB7
:102F9000D76FDA6BB60ED96FDC6BB80EDB6FDE6BFA
:102FA000BA0EDD6FE06BBB0EDF6FE26BBD0EE16F43
:102FB000E46BBF0EE36FE66BC10EE56FE86BC30E0B
:102FC000E76FEA6BC40EE96FEC6BC60EEB6FEE6B4E
:102FD000C80EED6FF06BCA0EEF6FF26BCB0EF16F98
:102FE000F46BCD0EF36FF66BCF0EF56FF86BD10E61
:102FF000F76FFA6BD30EF96FFC6BD40EFB6FFE6BA1
:10300000D60EFD6F0801006BD80E0701FF6F080197
:10301000026BDA0E016F046BDB0E036F066BDD0EC5
:10302000056F086BDF0E076F0A6BE10E096F0C6B03
:10303000E30E0B6F0E6BE40E0D6F106BE60E0F6F51
:10304000126BE80E116F146BEA0E136F166BEB0E1A
:10305000156F186BED0E176F1A6BEF0E196F1C6B57
:10306000F10E1B6F1E6BF30E1D6F206BF40E1F6FA6
:10307000226BF60E216F246BF80E236F266BFA0E6F
:10308000256F286BFB0E276F2A6BFD0E296F2C6BAB
:103090002B69010E2E6F2D6F306F030E2F6F010EF7
:1030A000326F040E316F010E346F060E336F010E56
:1030B000366F080E356F010E386F0A0E376F010E2E
:1030C0003A6F0B0E396F010E3C6F0D0E3B6F010E08
:1030D0003E6F0F0E3D6F010E406F110E3F6F010EE0
:1030E000426F130E416F010E446F140E436F010EB9
:1030F000466F160E456F010E486F180E476F010E92
:103100004A6F1A0E496F010E4C6F1B0E4B6F010E6A
:103110004E6F1D0E4D6F010E506F1F0E4F6F010E43
:10312000526F210E516F010E546F230E536F010E1B
:10313000566F240E556F010E586F260E576F010EF5
:103140005A6F280E596F010E5C6F2A0E5B6F010ECD
:103150005E6F2C0E5D6F010E606F2D0E5F6F010EA6
:10316000626F2F0E616F010E646F310E636F010E7F
:10317000666F330E656F010E686F340E676F010E58
:103180006A6F360E696F010E6C6F380E6B6F010E31
:103190006E6F3A0E6D6F010E706F3C0E6F6F010E09
:1031A000726F3D0E716F010E746F3F0E736F010EE3
:1031B000766F410E756F010E786F430E776F010EBB
:1031C0007A6F440E796F010E7C6F460E7B6F010E95
:1031D0007E6F480E7D6F010E806F4A0E7F6F010E6D
:1031E000826F4C0E816F010E846F4D0E836F010E46
:1031F000866F4F0E856F010E886F510E876F010E1F
:103200008A6F530E896F010E8C6F540E8B6F010EF7
:103210008E6F560E8D6F010E906F580E8F6F010ED0
:10322000926F5A0E916F010E946F5C0E936F010EA8
:10323000966F5D0E956F010E986F5F0E976F010E82
:103240009A6F610E996F010E9C6F630E9B6F030165
:10325000A06B3E0E9F6FA26B3F0EA16FA46B400E42
:10326000A36FA66B410EA56FA86B430EA76FAA6B49
:10327000440EA96FAC6B450EAB6FAE6B460EAD6FD7
:10328000B06B480EAF6FB26B490EB16FB46B4A0EA4
:10329000B36FB66B4B0EB56FB86B4D0EB76FBA6BA5
:1032A0004E0EB96FBC6B4F0EBB6FBE6B500EBD6F39
:1032B000C06B510EBF6FC26B530EC16FC46B540E07
:1032C000C36FC66B550EC56FC86B560EC76FCA6B02
:1032D000580EC96FCC6B590ECB6FCE6B5A0ECD6F9B
:1032E000D06B5B0ECF6FD26B5D0ED16FD46B5E0E69
:1032F000D36FD66B5F0ED56FD86B600ED76FDA6B5E
:10330000620ED96FDC6B630EDB6FDE6B640EDD6FFC
:10331000E06B650EDF6FE26B670EE16FE46B680ECA
:10332000E36FE66B690EE56FE86B6A0EE76FEA6BB9
:103330006B0EE96FEC6B6D0EEB6FEE6B6E0EED6F5F
:10334000F06B6F0EEF6FF26B700EF16FF46B720E2D
:10335000F36FF66B730EF56FF86B740EF76FFA6B15
:10336000750EF96FFC6B770EFB6FFE6B780EFD6FC1
:103370000401006B790E0301FF6F0401026B7A0EEA
:10338000016F046B7C0E036F066B7D0E056F086B7F
:103390007E0E076F0A6B7F0E096F0C6B810E0B6F31
:1033A0000E6B820E0D6F106B830E0F6F126B840EFF
:1033B000116F146B850E136F166B870E156F186BDC
:1033C000880E176F1A6B890E196F1C6B8A0E1B6F94
:1033D0001E6B8C0E1D6F206B8D0E1F6F226B8E0E61
:1033E000216F246B8F0E236F266B910E256F286B38
:1033F000920E276F2A6B930E296F2C6B940E2B6FF6
:103400002E6B960E2D6F306B970E2F6F326B980EC2
:10341000316F346B990E336F366B9B0E356F386B93
:103420009C0E376F3A6B9D0E396F3C6B9E0E3B6F57
:103430003E6B9F0E3D6F406BA10E3F6F426BA20E25
:10344000416F446BA30E436F466BA40E456F486BF0
:10345000A60E476F4A6BA70E496F4C6BA80E4B6FB9
:103460004E6BA90E4D6F506BAB0E4F6F526BAC0E87
:10347000516F546BAD0E536F566BAE0E556F586B4C
:10348000B00E576F5A6BB10E596F5C6BB20E5B6F1B
:103490005E6BB30E5D6F606BB50E5F6F626BB60EE9
:1034A000616F646BB70E636F666BB80E656F686BA8
:1034B000B90E676F6A6BBB0E696F6C6BBC0E6B6F7E
:1034C0006E6BBD0E6D6F706BBE0E6F6F726BC00E4C
:1034D000716F746BC10E736F766BC20E756F786B04
:1034E000C30E776F7A6BC50E796F7C6BC60E7B6FE0
:1034F0007E6BC70E7D6F806BC80E7F6F826BCA0EAE
:10350000816F846BCB0E836F866BCC0E856F886B5F
:10351000CD0E876F8A6BCF0E896F8C6BD00E8B6F41
:103520008E6BD10E8D6F906BD20E8F6F926BD30E10
:10353000916F946BD50E936F966BD60E956F986BBB
:10354000D70E976F9A6BD80E996F9C6BDA0E9B6FA4
:103550000801A06B740E9F6FA26B750EA16FA46B18
:10356000A36FA66B760EA56FA86B770EA76FAA6BDD
:10357000780EA96FAC6B790EAB6FAE6BAD6FB06BA5
:103580007A0EAF6FB26B7B0EB16FB46B7C0EB36F04
:10359000B66B7D0EB56FB86BB76FBA6B7E0EB96F39
:1035A000BC6B7F0EBB6FBE6B800EBD6FC06B810EA0
:1035B000BF6FC26B820EC16FC46BC36FC66B830ECD
:1035C000C56FC86B840EC76FCA6B850EC96FCC6B95
:1035D000860ECB6FCE6BCD6FD06B870ECF6FD26B5D
:1035E000880ED16FD46B890ED36FD66B8A0ED56FD0
:1035F000D86BD76FDA6B8B0ED96FDC6B8C0EDB6FF1
:10360000DE6B8D0EDD6FE06B8E0EDF6FE26B8F0E6B
:10361000E16FE46BE36FE66B900EE56FE86B910E84
:10362000E76FEA6B920EE96FEC6B930EEB6FEE6B4C
:10363000ED6FF06B940EEF6FF26B950EF16FF46B14
:10364000960EF36FF66B970EF56FF86BF76FFA6BDC
:10365000980EF96FFC6B990EFB6FFE6B9A0EFD6F67
:103660000901006B9B0E0801FF6F0901026B9C0EA4
:10367000016F046B036F066B9D0E056F086B9E0E4A
:10368000076F0A6B9F0E096F0C6BA00E0B6F0E6B12
:103690000D6F106BA10E0F6F126BA20E116F146BDA
:1036A000A30E136F166BA40E156F186B176F1A6BA2
:1036B000A50E196F1C6BA60E1B6F1E6BA70E1D6F40
:1036C000206BA80E1F6F226BA90E216F246B236F36
:1036D000266BAA0E256F286BAB0E276F2A6BAC0EDC
:1036E000296F2C6BAD0E2B6F2E6B2D6F306BAE0ECA
:1036F0002F6F326BAF0E316F346BB00E336F366B92
:10370000B10E356F386B376F3A6BB20E396F3C6B59
:10371000B30E3B6F3E6BB40E3D6F406BB50E3F6F0B
:10372000426BB60E416F446B436F466BB70E456FED
:10373000486BB80E476F4A6BB90E496F4C6BBA0EA7
:103740004B6F4E6B4D6F506BBB0E4F6F526BBC0E81
:10375000516F546BBD0E536F566BBE0E556F586B49
:10376000576F5A6BBF0E596F5C6BC00E5B6F5E6B11
:10377000C10E5D6F606BC20E5F6F626BC30E616FD7
:10378000646B636F666BC40E656F686BC50E676FA5
:103790006A6BC60E696F6C6BC70E6B6F6E6B6D6F6D
:1037A000706BC80E6F6F726BC90E716F746BCA0E3F
:1037B000736F766BCB0E756F786B776F7A6BCC0E01
:1037C000796F7C6BCD0E7B6F7E6BCE0E7D6F806BC9
:1037D000CF0E7F6F826BD00E816F846B836F866B91
:1037E000D10E856F886BD20E876F8A6BD30E896F6F
:1037F0008C6BD40E8B6F8E6B8D6F906BD50E8F6F25
:10380000926BD60E916F946BD70E936F966BD80E0A
:10381000956F986B976F9A6BD90E996F9C6BDA0EB8
:103820009B6FA06B650E9F6FA26B660EA16FA46B62
:10383000A36FA66B670EA56FA86BA76FAA6B680E28
:10384000A96FAC6B690EAB6FAE6BAD6FB06B6A0EF0
:10385000AF6FB26B6B0EB16FB46BB36FB66B6C0EB8
:10386000B56FB86BB76FBA6B6D0EB96FBC6B6E0E80
:10387000BB6FBE6BBD6FC06B6F0EBF6FC26BC16F96
:10388000C46B700EC36FC66B710EC56FC86BC76F0C
:10389000CA6B720EC96FCC6B730ECB6FCE6BCD6FD4
:1038A000D06B740ECF6FD26BD16FD46B750ED36F9C
:1038B000D66B760ED56FD86BD76FDA6B770ED96F64
:1038C000DC6B780EDB6FDE6BDD6FE06B790EDF6F2C
:1038D000E26BE16FE46B7A0EE36FE66B7B0EE56FF4
:1038E000E86BE76FEA6B7C0EE96FEC6BEB6FEE6BEE
:1038F0007D0EED6FF06B7E0EEF6FF26BF16FF46B80
:103900007F0EF36FF66B800EF56FF86BF76FFA6B47
:10391000810EF96FFC6BFB6FFE6B820EFD6F0A016F
:10392000006B830E0901FF6F0A01026B016F046BCC
:10393000840E036F066B850E056F086B076F0A6BAD
:10394000860E096F0C6B0B6F0E6B870E0D6F106B75
:10395000880E0F6F126B116F146B890E136F166B3D
:10396000156F186B8A0E176F1A6B8B0E196F1C6B05
:103970001B6F1E6B8C0E1D6F206B8D0E1F6F226BCD
:10398000216F246B8E0E236F266B256F286B8F0E95
:10399000276F2A6B900E296F2C6B2B6F2E6B910E5D
:1039A0002D6F306B920E2F6F326B316F346B930E25
:1039B000336F366B356F386B940E376F3A6B950EED
:1039C000396F3C6B3B6F3E6B960E3D6F406B3F6FAC
:1039D000426B970E416F446B980E436F466B456F79
:1039E000486B990E476F4A6B9A0E496F4C6B4B6F41
:1039F0004E6B9B0E4D6F506B4F6F526B9C0E516F09
:103A0000546B9D0E536F566B556F586B9E0E576FD0
:103A10005A6B9F0E596F5C6B5B6F5E6BA00E5D6F98
:103A2000606B5F6F626BA10E616F646BA20E636F60
:103A3000666B656F686BA30E676F6A6B696F6C6B03
:103A4000A40E6B6F6E6BA50E6D6F706B6F6F726BEC
:103A5000A60E716F746BA70E736F766B756F786BB4
:103A6000A80E776F7A6B796F7C6BA90E7B6F7E6B7C
:103A7000AA0E7D6F806B7F6F826BAB0E816F846B44
:103A8000AC0E836F866B856F886BAD0E876F8A6B0C
:103A9000896F8C6BAE0E8B6F8E6BAF0E8D6F906BD4
:103AA0008F6F926BB00E916F946B936F966BB10E9C
:103AB000956F986BB20E976F9A6B996F9C6BB30E64
:103AC0009B6FA06B8C0E9F6FA26B8D0EA16FA46B72
:103AD0008E0EA36FA66B8F0EA56FA86BA76FAA6B38
:103AE000900EA96FAC6B910EAB6FAE6B920EAD6F7B
:103AF000B06BAF6FB26B930EB16FB46B940EB36FCC
:103B0000B66B950EB56FB86B960EB76FBA6BB96F93
:103B1000BC6B970EBB6FBE6B980EBD6FC06B990EE2
:103B2000BF6FC26BC16FC46B9A0EC36FC66B9B0E27
:103B3000C56FC86B9C0EC76FCA6B9D0EC96FCC6BEF
:103B4000CB6FCE6B9E0ECD6FD06B9F0ECF6FD26BB7
:103B5000A00ED16FD46BD36FD66BA10ED56FD86B7F
:103B6000A20ED76FDA6BA30ED96FDC6BDB6FDE6B47
:103B7000A40EDD6FE06BA50EDF6FE26BA60EE16FAA
:103B8000E46BA70EE36FE66BE56FE86BA80EE76FDB
:103B9000EA6BA90EE96FEC6BAA0EEB6FEE6BED6FA3
:103BA000F06BAB0EEF6FF26BAC0EF16FF46BAD0E12
:103BB000F36FF66BAE0EF56FF86BF76FFA6BAF0E37
:103BC000F96FFC6BB00EFB6FFE6BB10EFD6F0B015E
:103BD000006B0A01FF6F0B01026BB20E016F046BE9
:103BE000B30E036F066BB40E056F086BB50E076F4F
:103BF0000A6B096F0C6BB60E0B6F0E6BB70E0D6F69
:103C0000106BB80E0F6F126B116F146BB90E136F30
:103C1000166BBA0E156F186BBB0E176F1A6B196FF8
:103C20001C6BBC0E1B6F1E6BBD0E1D6F206BBE0E82
:103C30001F6F226BBF0E216F246B236F266BC00E8C
:103C4000256F286BC10E276F2A6BC20E296F2C6B54
:103C50002B6F2E6BC30E2D6F306BC40E2F6F326B1C
:103C6000C50E316F346BC60E336F366B356F386BE4
:103C7000C70E376F3A6BC80E396F3C6BC90E3B6F7E
:103C80003E6B3D6F406BCA0E3F6F426BCB0E416F78
:103C9000446BCC0E436F466B456F486BCD0E476F40
:103CA0004A6BCE0E496F4C6BCF0E4B6F4E6BD00EE6
:103CB0004D6F506B4F6F526BD10E516F546BD20ED4
:103CC000536F566BD30E556F586B576F5A6BD40E9C
:103CD000596F5C6BD50E5B6F5E6BD60E5D6F606B64
:103CE000D70E5F6F626B616F646BD80E636F666B2C
:103CF000D90E656F686BDA0E676F6A6B696F6C6BF4
:103D0000DB0E6B6F6E6BDC0E6D6F706BDD0E6F6FAD
:103D1000726BDE0E716F746B736F766BDF0E756F87
:103D2000786BE00E776F7A6BE10E796F7C6B7B6F4F
:103D30007E6BE20E7D6F806BE30E7F6F826BE40E15
:103D4000816F846B836F866BE50E856F886BE60EE3
:103D5000876F8A6BE70E896F8C6BE80E8B6F8E6BAB
:103D60008D6F906BE90E8F6F926BEA0E916F946B73
:103D7000EB0E936F966B956F986BEC0E976F9A6B3B
:103D8000ED0E996F9C6BEE0E9B6FA06B7E0E9F6F7E
:103D9000A26BA16FA46B7F0EA36FA66BA56FA86B20
:103DA000800EA76FAA6BA96FAC6B810EAB6FAE6B69
:103DB000AD6FB06B820EAF6FB26BB16FB46B830E31
:103DC000B36FB66BB56FB86B840EB76FBA6BB96F64
:103DD000BC6B850EBB6FBE6BBD6FC06B860EBF6FBD
:103DE000C26BC16FC46B870EC36FC66BC56FC86BE8
:103DF000880EC76FCA6BC96FCC6B890ECB6FCE6B49
:103E0000CD6FD06B8A0ECF6FD26BD16FD46B8B0E10
:103E1000D36FD66BD56FD86B8C0ED76FDA6BD96F2B
:103E2000DC6B8D0EDB6FDE6BDD6FE06B8E0EDF6F9C
:103E3000E26BE16FE46B8F0EE36FE66BE56FE86BAF
:103E4000900EE76FEA6BE96FEC6B910EEB6FEE6B28
:103E5000ED6FF06B920EEF6FF26BF16FF46B930EF0
:103E6000F36FF66BF56FF86B940EF76FFA6BF96FF3
:103E7000FC6B950EFB6FFE6BFD6F0C01006B960EDD
:103E80000B01FF6F0C01026B016F046B970E036F48
:103E9000066B056F086B980E076F0A6B096F0C6B4A
:103EA000990E0B6F0E6B0D6F106B9A0E0F6F126BDE
:103EB000116F146B9B0E136F166B156F186B9C0EA6
:103EC000176F1A6B196F1C6B9D0E1B6F1E6B1D6F8E
:103ED000206B9E0E1F6F226B216F246B9F0E236F32
:103EE000266B256F286BA00E276F2A6B296F2C6B12
:103EF000A10E2B6F2E6B2D6F306BA20E2F6F326BBE
:103F0000316F346BA30E336F366B356F386BA40E85
:103F1000376F3A6B396F3C6BA50E3B6F3E6B3D6F55
:103F2000406BA60E3F6F426B416F446BA70E436F11
:103F3000466B456F486BA80E476F4A6B496F4C6BD9
:103F4000A90E4B6F4E6B4D6F506BAA0E4F6F526B9D
:103F5000516F546BAB0E536F566B556F586BAC0E65
:103F6000576F5A6B596F5C6BAD0E5B6F5E6B5D6F1D
:103F7000606BAE0E5F6F626B616F646BAF0E636FF1
:103F8000666B656F686BB00E676F6A6B696F6C6BA1
:103F9000B10E6B6F6E6B6D6F706BB20E6F6F726B7D
:103FA000716F746BB30E736F766B756F786BB40E45
:103FB000776F7A6B796F7C6BB50E7B6F7E6B7D6FE5
:103FC000806BB60E7F6F826B816F846BB70E836FD1
:103FD000866B856F886BB80E876F8A6B896F8C6B69
:103FE000B90E8B6F8E6B8D6F906BBA0E8F6F926B5D
:103FF000916F946BBB0E936F966B956F986BBC0E25
:10400000976F9A6B996F9C6BBD0E9B6FA06B6A0E3E
:104010009F6FA26BA16FA46B6B0EA36FA66BA56FB6
:10402000A86B6C0EA76FAA6B6D0EA96FAC6BAB6F14
:10403000AE6B6E0EAD6FB06BAF6FB26B6F0EB16FDC
:10404000B46BB36FB66B700EB56FB86BB76FBA6BFE
:10405000710EB96FBC6BBB6FBE6B720EBD6FC06B68
:10406000730EBF6FC26BC16FC46B740EC36FC66B30
:10407000C56FC86B750EC76FCA6BC96FCC6B760EF8
:10408000CB6FCE6BCD6FD06B770ECF6FD26BD16F06
:10409000D46B780ED36FD66BD56FD86B790ED76F84
:1040A000DA6B7A0ED96FDC6BDB6FDE6B7B0EDD6F4C
:1040B000E06BDF6FE26B7C0EE16FE46BE36FE66B4E
:1040C0007D0EE56FE86BE76FEA6B7E0EE96FEC6BD8
:1040D000EB6FEE6B7F0EED6FF06B800EEF6FF26BA0
:1040E000F16FF46B810EF36FF66BF56FF86B820E68
:1040F000F76FFA6BF96FFC6B830EFB6FFE6BFD6F56
:104100000D01006B840E0C01FF6F0D01026B016F3E
:10411000046B850E036F066B056F086B860E076FC9
:104120000A6B870E096F0C6B0B6F0E6B880E0D6F91
:10413000106B0F6F126B890E116F146B136F166B70
:104140008A0E156F186B176F1A6B8B0E196F1C6B1D
:104150001B6F1E6B8C0E1D6F206B8D0E1F6F226BE5
:10416000216F246B8E0E236F266B256F286B8F0EAD
:10417000276F2A6B296F2C6B900E2B6F2E6B2D6F78
:10418000306B910E2F6F326B316F346B920E336F39
:10419000366B356F386B930E376F3A6B940E396F01
:1041A0003C6B3B6F3E6B950E3D6F406B3F6F426BC0
:1041B000960E416F446B436F466B970E456F486B8D
:1041C000476F4A6B980E496F4C6B4B6F4E6B990E55
:1041D0004D6F506B9A0E4F6F526B516F546B9B0E1D
:1041E000536F566B556F586B9C0E576F5A6B596FC8
:1041F0005C6B9D0E5B6F5E6B5D6F606B9E0E5F6FA9
:10420000626B616F646B9F0E636F666B656F686B4B
:10421000A00E676F6A6BA10E696F6C6B6B6F6E6B34
:10422000A20E6D6F706B6F6F726BA30E716F746BFC
:10423000736F766BA40E756F786B776F7A6BA50EC4
:10424000796F7C6B7B6F7E6BA60E7D6F806BA70E8C
:104250007F6F826B816F846BA80E836F866B856F17
:10426000886BA90E876F8A6B896F8C6BAA0E8B6F18
:104270008E6B8D6F906BAB0E8F6F926B916F946B9B
:10428000AC0E936F966B956F986BAD0E976F9A6BA4
:0E429000AE0E996F9C6B9B6F00011200FFD762
:020000040030CA
:0300010006160ED2
:020005008580F4
:060008000FC00FE00F40E5
:00000001FF
